:100000000C9446000C947C000C947C000C947C00B6
:100010000C947C000C947C000C947C000C947C0070
:100020000C947C000C947C000C947C000C947C0060
:100030000C947C000C947C000C947C000C947C0050
:100040000C947C000C947C000C947C000C947C0040
:100050000C947C000C947C000C947C000C947C0030
:100060000C947C000C947C000C947C000C947C0020
:100070000C947C000C947C000C947C000C947C0010
:100080000C947C000C947C000C947C0011241FBE0A
:10009000CFEFD0E1DEBFCDBF0E9452000C945000E4
:0400A000F894FFCF02
:1000A4008FEF81BB81E082BBC0E082B3803809F46A
:1000B400C1E082B3813009F4C0E0C11104C082B34D
:1000C400880F82BB03C082B3869582BB80E590E033
:0600D4000E946D00EACF5E
:1000DA0020E030E008C0E3ECF9E03197F1F700C026
:0E00EA0000002F5F3F4F28173907ACF3089531
:0400F8000C94000064
:00000001FF
